:020000008A284C
:10000800A000030E8301BA000A08B50003308A0075
:10001800732B03178D0083168C130C1483120C0892
:10002800852803178C0083168C130C1555308D000A
:10003800AA308D008C148C181F280C118528A40157
:10004800A300FF30A307031CA407031C8528033063
:10005800A200DF3031202528A201E83EA100A20934
:10006800FC30031C3A28A10703183728A1076400AD
:10007800A20F372821184028A11C44280000442832
:100088000800A201A401A30002305428A201A4017F
:10009800A30006305428A201A401A3000430542868
:1000A800A90024082202031D5B282308210204302A
:1000B80003180130031902302905031DFF30852874
:1000C8000038031DFF300405031DFF308528040494
:1000D800031DFF3085281030A900A201A101A80C3A
:1000E800A70C031C7D282308A10724080318240F44
:1000F800A207A20CA10CA60CA50CA90B7328250815
:10010800852883130313831264000800F5018A11FC
:100118004E2C64005908073C8A11031DA928013098
:100128005A07CC00CD01CD0D4C08A7004D08A800FA
:100138001630A300A4018A016F20CC002608CD0048
:100148004D08A4004C088A01242064005908083C82
:100158008A11031DC52801305A07CC00CD01CD0DE9
:100168004C08A7004D08A8001030A300A4018A017C
:100178006F20CC002608CD004D08A4004C088A0149
:1001880024205908A10009308A014520CC005908CB
:10019800A10005308A014520CE004C0884004E0895
:1001A8008A016B20CE00CF005908A10004308A01D3
:1001B8004520D0004E084F04840050088A016B2067
:1001C800D000D1006400500851048A110319022993
:1001D80001305A07CC00CD01CD0D4C08A7004D08C1
:1001E800A8000C30A300A4018A016F20CC002608C7
:1001F800CD004D08A4004C088A01242008006A0894
:10020800193C8A11031C2B298A110D21E8008A1137
:100218002B2901308A006A088207EC34F1349C34B7
:10022800F1349C348C34BC346C34913478340C34D0
:100238001C346E346E34FC34CC34FC34CC34B434DA
:1002480081347C340C346C340234023490346A08BF
:10025800193C8A11031C53298A113521E9008A1196
:10026800532901308A006A08820744345034003424
:100278001034443404344034443410340034A43446
:10028800003480342034003444342034643444341A
:100298001034003488342834A834883488348A11D7
:1002A800BB2C6A08093C8A11031C6D298A115F213D
:1002B800E8008A116D2901308A006A088207FC3437
:1002C8006034D834F0346434B434BC34E034FC34AE
:1002D800E4346A08093C8A11031C85298A117721AC
:1002E800E9008A11852901308A006A088207883462
:1002F80000344434443444344434443400344434BE
:1003080044348A11BB2C6A08093C8A11031C9F29B2
:100318008A119121E8008A119F2901308A006A0810
:100328008207FC340134D034B03404349434BC34FF
:1003380080341E34E4346A08093C8A11031CB72946
:100348008A11A921E9008A11B72901308A006A08AF
:100358008207883410344834C0348C34243444340C
:100368009034243444348A11BB2C6A08093C8A111D
:10037800031CD1298A11C321E8008A11D12901302F
:100388008A006A0882077034003490349034043448
:10039800923410348034923482346A08093C8A11C9
:1003A800031CE9298A11DB21E9008A11E9290130B6
:1003B8008A006A088207883488348834A0348C34E8
:1003C8002034A8348834A83488348A11BB2C6A08AD
:1003D800093C8A11031C0B2A8A11F521E8008A11AD
:0A03E8000B2A02308A006A08002A7E
:1004000082071E346034983490340434B23430346B
:100410008034B43484346A08093C8A11031C232ACA
:100420008A111522E9008A11232A02308A006A08FB
:100430008207203480348434A43494344034C83463
:100440009034CC3494348A11BB2C6A08093C8A114C
:10045000031C3D2A8A112F22E8008A113D2A02300E
:100460008A006A088207FC346034D834F034663479
:10047000B634BC34C034FE34E4346A08093C8A1112
:10048000031C552A8A114722E9008A11552A023095
:100490008A006A088207A834C034CC34E034E434DB
:1004A00064346C34D0344C34A4348A11BB2C6A08C4
:1004B000093C8A11031C6F2A8A116122E8008A1103
:1004C0006F2A02308A006A088207FC3400346E34D6
:1004D000FD3491346C346C349C34FD349D346A08A2
:1004E000093C8A11031C872A8A117922E9008A11A2
:1004F000872A02308A006A08820744344434483428
:1005000010341434A434E4340034543414348A11D0
:10051000BB2C6A08093C8A11031CA12A8A11932268
:10052000E8008A11A12A02308A006A088207FC3496
:10053000603416349234063450348C34813426348A
:1005400016346A08093C8A11031CB92A8A11AB22A5
:10055000E9008A11B92A02308A006A088207283421
:10056000A0340C340C345434E0340C3490346434FF
:1005700024348A11BB2C6A08093C8A11031CD32A33
:100580008A11C522E8008A11D32A02308A006A083B
:1005900082076E340F340E340E340E3460346034FF
:1005A0006034623461346A08093C8A11031CEB2A06
:1005B0008A11DD22E9008A11EB2A02308A006A08DA
:1005C0008207A8340834883448342834B034A83436
:1005D000A434A034A0348A11BB2C6A08093C8A11C7
:1005E000031C0B2B8A11F722E8008A110B2B033016
:0605F0008A006A08002BDE
:1006000082078034C034E034F034F834FC34FE34F3
:10061000FF34FF34FF346A08093C8A11031C232B82
:100620008A111523E9008A11232B03308A006A08F6
:1006300082070034003400340034003400340034C5
:1006400000348034C0348A11BB2C6A08093C8A11FA
:10065000031C3D2B8A112F23E8008A113D2B033008
:100660008A006A0882078034403420341034083409
:10067000043402340134003400346A08093C8A111D
:10068000031C552B8A114723E9008A11552B03308F
:100690008A006A08820700340034003400340034D1
:1006A000003400340034803440348A11BB2C6400A0
:1006B0007E306A028A11031C5F2B8A11BB2C6A08E8
:1006C000A700A8010230A300A4018A016F20D7006F
:1006D00057088A010D20E800D70A57088A010D2023
:1006E000E9008A11BB2C0B1F3F2C8C1E3F2C1A08D3
:1006F000EE00990000000C1E7B2B6D18852B6D14ED
:100700006E08243A031D3A2C472CED188D2BED145E
:100710006E08423A031D3A2C472C6D19952B6D1526
:100720006E08373A031D3A2C472CED19C52BED15F1
:10073000EF016E08F0004D3A0319B32B7008463AEA
:100740000319B92B7008573A0319B62B7008453AAC
:100750000319BC2B7008533A0319BF2B7008553A84
:100760000319C22B3A2C0130F400472C0230F4005C
:10077000472C0330F400472C0430F400472C05309C
:10078000F400472C0730F400472C6E080D3A03198B
:10079000E62B7408023A031DDB2B11306F0203189D
:1007A000472C3B306F0784006E0880006F08FF3ACB
:1007B000031DEF0A472C6F08FF3A031DEF0A6F086D
:1007C0005506031D472C6E08EA00472C55086F029A
:1007D000031C3A2C6A08213A03193A2C7408033A8C
:1007E000031DFB2B6A08DB003030DB025B08D800FE
:1007F000FD30D700152C7408043A031D082C6A0834
:10080000D9003030D9025908D800FE30D700152C55
:100810007408053A031D2B2C6A08DA003030DA021E
:100820005A08D800FF30D700152C831203130D127D
:10083000570803178D000313580803178C008316FD
:100840008C130C1555308D00AA308D008C140000CF
:10085000831203133A2C7408073A031D382C6A08D4
:10086000303A0319F5136A08313A0319F5173A2C8F
:10087000D414472CEF01F401ED01D410472C0B1DCB
:10088000472C0B11F20B472C54147308F200350857
:100890008A003A0E8300A00E200E090083168730CE
:1008A0009F00850120308600870183128501860123
:1008B00087018B0183168C0187308100831294019C
:1008C00083169401831203179E019F01831603135D
:1008D0009B018312831690011830990061308F00BC
:1008E000A43098008312903098001830F3007308F9
:1008F000F200EF01D3010130D600F5012030EA000B
:10090000D401F401E201E301E801E901DB01013076
:10091000D9000330DA000C1E8B2CAB30990000009C
:100920000C1E902C01308A01232018121A081A0874
:100930001A08181600000000AB30990000000C1EC9
:100940009F2C05308A0123201A08AB3A0319B02CDA
:100950000130D500EA00990000000C1EAD2C042ED9
:100960008C1EB02C1A08013ED500990000000C1E08
:10097000B72C8A11042EE81B6214E81F6210681B52
:100980006414681F6410E81A6215E81E6211681A80
:10099000E216681EE212E8196416E81D641268196E
:1009A000E415681DE411E8186417E81C641368185E
:1009B0006317681C6313E91BE414E91FE410691B47
:1009C000E214691FE210E91A6415E91E6411691A3C
:1009D0006216691E6212E919E417E91DE413691928
:1009E000E416691DE412E9186316E91C6312F51B8D
:1009F00063168A11DF2EED01D4108316D410640023
:100A000083127408003C8A110319082D8A110B2DDA
:100A1000EF01F40108007308F20064007408023C5E
:100A20008A1103193A2DF40164005B08253C8A11F0
:100A30000319352D2F30A1006A088A014F20CC0000
:100A40006A08A1003A308A014F20CE004C08840089
:100A50004E088A016420CE00CF0064004E084F0487
:100A60008A110319352D3030EA02D4178316D413B6
:100A70008312080064005B08253C8A110319412D8C
:100A80000800F40164007E303B028A11031C492DEA
:100A900008003B08A700A8010230A300A4018A01B6
:100AA0006F20D700D80164003C08313C8A11031D37
:100AB0005D2DD8178316D813831264003D08313C8E
:100AC0008A11031D672D581783165813831264006B
:100AD0003E08313C8A11031D712DD8168316D81299
:100AE000831264003F08313C8A11031D7B2D581688
:100AF00083165812831264004008313C8A11031D8A
:100B0000852DD8158316D811831264004108313C15
:100B10008A11031D8F2D58158316581183126400F6
:100B20004208313C8A11031D992DD8148316D81020
:100B3000831264004308313C8A11031DA32D58140D
:100B4000831658108312570803178D000313580893
:100B50008A011520D70AD80164004408313C8A1163
:100B6000031DB62DD8178316D813831264004508C9
:100B7000313C8A11031DC02D581783165813831258
:100B800064004608313C8A11031DCA2DD81683160D
:100B9000D812831264004708313C8A11031DD42DFA
:100BA000581683165812831264004808313C8A1183
:100BB000031DDE2DD8158316D81183126400490851
:100BC000313C8A11031DE82D5815831658118312E4
:100BD00064004A08313C8A11031DF22DD814831693
:100BE000D810831264004B08313C8A11031DFC2D80
:100BF0005814831658108312570803178D000313D7
:100C000058088A0115200800FD308A010D20DB00FC
:100C1000FE308A010D20D900FF308A010D20DA0054
:100C2000E0308B00831620308C00831264008A1120
:100C3000541C1E2E541083165410831264008A1103
:100C4000D41C242E8A01FB2464008A11D41F2A2E6E
:100C50008A112C268A01162ED4138316D4138312DC
:100C6000A1016A088A014A20CC006A08A1000A3062
:100C70008A014F20CE004C0884004E088A0164206F
:100C8000CE00CF0064004E084F048A1103194A2E8B
:100C90008A117B2E64005B08253C8A11031D522EAD
:100CA0008A01572B4030A1006A088A014F20CC00EE
:100CB0006A08A1005B308A014F20CE004C088400F6
:100CC0004E088A016420CE00CF0064004E084F0415
:100CD0008A1103196F2E4130EA028A010329640048
:100CE0006A08203C8A11031D792EE801E9018A0176
:100CF000BB2C8A15632864005B08003C8A11031D25
:100D0000852E8A0155298A11DD2E64005B08013C7D
:100D10008A11031D8F2E8A0187298A11DD2E640016
:100D20005B08023C8A11031D992E8A01B9298A1198
:100D3000DD2E64005B08033C8A11031DA32E8A018B
:100D4000EB298A11DD2E64005B08043C8A11031D27
:100D5000AD2E8A01252A8A11DD2E64005B08053C30
:100D60008A11031DB72E8A01572A8A11DD2E6400CD
:100D70005B08063C8A11031DC12E8A01892A8A114B
:100D8000DD2E64005B08073C8A11031DCB2E8A010F
:100D9000BB2A8A11DD2E64005B08083C8A11031D02
:100DA000D52E8A01ED2A8A11DD2E64005B08093CEC
:100DB0008A11031DDD2E8A01252B8A015529590828
:100DC000A200093C8A11031C152FA20D8A11EF26DF
:100DD000A10022108A11EF268A0021088200073024
:060DE0008A002208002F2A
:100E000082070834633408346B3408346B34083494
:100E1000C3340C343A340D3462340A34F0340734B9
:100E20001734073417340934DA348A1563288714E1
:100E3000831687108312871783168713831206136E
:100E400083160613831205128316051283120510EA
:100E500083160510831285128316851283120612DB
:100E60008316061283128A018D208514831685103D
:100E700083128716831687128312871083168710B2
:100E800083128713831687138312071083160710A4
:100E9000831207128316071283128A018D20071509
:100EA0008316071183120717831607138312851001
:100EB00083168510831287128316871283120511F9
:100EC00083160511831287118316871183128A01F5
:100ED0008D20051683160512831206178316061336
:100EE0008312071183160711831207138316071342
:100EF00083128A018D2064005908083C8A11031965
:100F0000832F8A11CB2F871483168710831287179C
:100F10008316871383120613831606138312051292
:100F20008316051283128A018D208514831685107D
:100F300083128716831687128312871083168710F1
:100F4000831287138316871383128A018D20071556
:100F50008316071183120717831607138312851050
:100F600083168510831287128316871283128A01D3
:100F70008D20051683160512831206178316061395
:100F800083120711831607118312071383160713A1
:100F900083128A018D208714831687108312871786
:100FA0008316871364008A118312691ADB2F0512D6
:100FB00083160512831264008A116818E32F061342
:100FC0008316061383128A018D20851483168510DB
:100FD000831287168316871264008A118312E91B15
:100FE000F52F871083168710831264008A11E91980
:100FF000FD2F871383168713831264008A15681FD9
:101000000528071483160710831264008A15E81D4B
:101010000D2807168316071283128A018D200715E3
:1010200083160711831207178316071364008A15A6
:101030008312691B1F288510831685108312640094
:101040008A1569192728871283168712831264006C
:101050008A15E81E2F2805158316051183126400D2
:101060008A15681D372887158316871183128A0110
:101070008D2064008A15E91A41280711831607118B
:10108000831264008A15E81849280713831607138A
:10109000831264008A15E81F512805148316051071
:1010A000831264008A15681E5928851683168512D6
:1010B000831264008A15F51F61280616831606122E
:1010C00083128A1554296408870063088600620821
:1010D00085008A1554295A0AD200DC015208A7005B
:1010E000A8011930A300A4018A016F20DE0064006A
:1010F0005908023C8A15031D86285208A700A8013A
:101100001530A300A4018A016F20DE00DC01640019
:101110005C085E028A15031CBB28DD01DD0164004A
:1011200009305D028A150318B72862088500630834
:101130008600640887005908023A031DA2285E0849
:10114000DF00A5285C08013EDF00DF0BA52865084D
:10115000850066088600670887005C085E02013E1D
:10116000DF00DF0BB128DD0A8A15031D8F28DC0A9A
:101170008A15031D872862088500630886006408B5
:1011800087008A1554295A0AD200DC015208A700A8
:10119000A8011930A300A4018A016F20DE006400B9
:1011A0005908043C8A15031DDE285208A700A8012F
:1011B0000F30A300A4018A016F20DE00DC0164006F
:1011C0005C085E028A15031C0C29DD01DD01640048
:1011D0000A305D028A1503180829FF308500EF30B8
:1011E0008600FF3087005C08013EDF00DF0BF62839
:1011F0006508850066088600670887005C085E024F
:10120000013EDF00DF0B0229DD0A8A15031DE728F6
:10121000DC0A8A15031DDF2864005908053C8A157D
:10122000031D14298A154C29DC015208A700A801C6
:101230001930A300A4018A016F20DE00DC016400E4
:101240005C085E028A15031C4C29DD01DD01640087
:1012500007305D028A150318482962088500630873
:101260008600640887005C08013EDF00DF0B36293A
:10127000FF308500EF308600FF3087005C085E029B
:10128000013EDF00DF0B4229DD0A8A15031D2729F5
:10129000DC0A8A15031D1F29620885006308860081
:1012A000640887008A1554296208E5006308E6008F
:1012B0006408E70008000508E5005A0AD200DC01CE
:1012C0005208A700A8011930A300A4018A016F20C9
:1012D000DE00DC0164005C085E028A15031C8329C1
:1012E000710885005C08013EDF00DF0B7529650889
:1012F00085005C085E02013EDF00DF0B7D29DC0A11
:101300008A15031D6A297108850008000608E60091
:101310005A0AD200DC015208A700A8011930A30024
:10132000A4018A016F20DE00DC0164005C085E021B
:101330008A15031CAC295C08013EDF00DF0B9E29E7
:10134000660886005C085E02013EDF00DF0BA6290E
:10135000DC0A8A15031D9529710886000800070814
:10136000E7005A0AD200DC015208A700A801193090
:10137000A300A4018A016F20DE00DC0164005C0888
:101380005E028A15031CD729710887005C08013E9C
:10139000DF00DF0BC929670887005C085E02013E99
:1013A000DF00DF0BD129DC0A8A15031DBE29710875
:1013B0008700080087148316871083120510831690
:1013C000051083128A018D208514831685108312DF
:1013D0008710831687108312071083160710831255
:1013E0008A018D2007158316071183128510831635
:1013F0008510831205118316051183128A018D2031
:10140000051683160512831207118316071183121E
:101410008A018D208717831687138312051283167E
:101420000512831285128316851283120612831603
:10143000061283128A018D20871683168712831263
:1014400087138316871383120712831607128312DA
:101450008A018D20071783160713831287128316BC
:101460008712831287118316871183128A018D20B8
:1014700006178316061383120713831607138312A6
:101480008A018D2087148316871064008A158312C1
:1014900068184E2A061383160613831264008A15F1
:1014A000E81F562A05148316051083128A018D2021
:1014B00085148316851064008A158312E91B642A3B
:1014C000871083168710831264008A15681F6C2AA0
:1014D00007148316071083128A018D2007158316BF
:1014E000071164008A158312691B7A2A85108316F6
:1014F0008510831264008A15E81E822A051583165A
:10150000051183128A018D200516831605126400C9
:101510008A158312E91A902A07118316071183127C
:101520008A018D2087178316871364008A1583121A
:10153000691A9E2A051283160512831264008A1501
:10154000681EA62A851683168512831264008A15E2
:10155000F51FAE2A06168316061283128A018D2005
:1015600087168316871264008A158312E919BC2A2C
:10157000871383168713831264008A15E81DC42A13
:1015800007168316071283128A018D200717831608
:10159000071364008A1583126919D22A87128316E9
:1015A0008712831264008A15681DDA2A871583164C
:1015B000871183128A018D2064008A15681CE42A31
:1015C000061783160613831264008A15E818EC2A9E
:1015D00007138316071383128A018D208A15542955
:1015E00064008A150518F62A8A15FA2A0503F100FF
:1015F0008A155B2164008A150519002B8A15052BB5
:1016000004300502F1008A155B2164008A15071970
:101610000B2B8A15102B04300702F1008A15AF211D
:1016200064008A15871A162B8A151B2B2030070297
:10163000F1008A15AF2164008A15061B212B8A153B
:10164000262B40300602F1008A15862164008A1597
:10165000051A2C2B8A15312B10300502F1008A1542
:101660005B2164008A158719372B8A153C2B0830BB
:101670000702F1008A15AF2164008A158518422BF4
:101680008A15472B02300502F1008A155B216400A0
:101690008A15851A4D2B8A15522B20300502F10030
:1016A0008A155B2164008A150718582B8A155C2B54
:1016B0000703F1008A15AF2164008A15871B622B8E
:1016C0008A15672B80300702F1008A15AF2164006C
:1016D0008A15071B6D2B8A15722B40300702F1000B
:1016E0008A15AF2164008A158718782B8A157D2BFF
:1016F00002300702F1008A15AF2164008A15071A2B
:10170000832B8A15882B10300702F1008A15AF2130
:1017100064008A15061A8E2B8A15932B1030060248
:10172000F1008A1586218A15952B64008A156218A6
:101730009B2B8A159F2B050AF1008A155B216400FB
:101740008A156219A52B8A15AA2B04300507F1000A
:101750008A155B2164008A156419B02B8A15B52B94
:1017600004300707F1008A15AF2164008A15E41AD6
:10177000BB2B8A15C02B20300707F1008A15AF213B
:1017800064008A15631BC62B8A15CB2B40300607D5
:10179000F1008A15862164008A15621AD12B8A15F8
:1017A000D62B10300507F1008A155B2164008A15DD
:1017B000E419DC2B8A15E12B08300707F1008A15A4
:1017C000AF2164008A15E218E72B8A15EC2B023052
:1017D0000507F1008A155B2164008A15E21AF22BD5
:1017E0008A15F72B20300507F1008A155B2164006C
:1017F0008A156418FD2B8A15012C070AF1008A1539
:10180000AF2164008A15E41B072C8A150C2C80304C
:101810000707F1008A15AF2164008A15641B122C9A
:101820008A15172C40300707F1008A15AF21640094
:101830008A15E4181D2C8A15222C02300707F100A6
:101840008A15AF2164008A15641A282C8A152D2C5C
:1018500010300707F1008A15AF2164008A15631A5A
:10186000332C8A15382C10300607F1008A15862192
:101870008A15542906178316061383128A018D20B0
:101880000717831607138312871483168710831292
:101890000613831606138312051083160510831290
:1018A0008A018D208716831687128312851483166A
:1018B00085108312871083168710831207138316EF
:1018C00007138312071083160710831287118316DC
:1018D000871183128A018D20071583160711831241
:1018E0008717831687138312871283168712831232
:1018F0008510831685108312071283160712831230
:1019000005118316051183128A018D200516831691
:101910000512831287138316871383120711831608
:101920000711831285128316851283128A018D2076
:1019300005128316051283120612831606128312ED
:101940008A018D2005168316051283128A018D20C7
:1019500064008A15F51FB02C061683160612831232
:1019600085168316851283120715831607118312B5
:1019700087178316871364008A158312691AC42C8B
:1019800005128316051283128A018D20871683168D
:10199000871283128514831685108312051583160A
:1019A0000511831207168316071264008A15831225
:1019B000E91ADE2C071183160711831264008A15B9
:1019C000E919E62C871383168713831264008A159E
:1019D000681AEE2C85128316851283128A018D20D7
:1019E0000717831607138312871483168710831231
:1019F0000714831607108312871583168711640056
:101A00008A1583126919082D87128316871283128B
:101A100064008A15691B102D8510831685108312AA
:101A200064008A15E81A182D051183160511831212
:101A300064008A15E819202D0712831607128312F5
:101A40008A018D2005148316051064008A158312FF
:101A5000681B2E2D071083160710831264008A1549
:101A60006819362D87118316871183128A018D20FC
:101A700006178316061364008A158312E91B442D8A
:101A8000871083168710831264008A15E8184C2D7E
:101A9000071383160713831264008A15E81B542D5D
:101AA00005108316051083128A018D2064008A15A3
:101AB00068185E2D06138316061383128A018D2083
:101AC0008A15542987168316871283128A018D205E
:101AD000871783168713831207178316071383123A
:101AE0008712831687128312871183168711831238
:101AF00007128316071283128A018D200617831698
:101B00000613831205168316051283128713831694
:101B10008713831207138316071383128A018D20FC
:101B200007158316071183128714831687108312F3
:101B300006138316061383120512831605128312E9
:101B400005108316051083128512831685128312E1
:101B500006128316061283128A018D2085148316BD
:101B6000851083128710831687108312071183163E
:101B700007118312071083160710831205118316AD
:101B8000051183128A018D2085108316851083121A
:101B90008A018D2087168316871283128A018D2071
:101BA000071683160712831287158316871183126F
:101BB000871783168713831207178316071364008A
:101BC0008A1583126919E82D8712831687128312EA
:101BD0008A018D20061783160613831205168316B5
:101BE000051264008A158312F51FFA2D0616831656
:101BF0000612831264008A15E919022E87138316D0
:101C00008713831264008A15E8180A2E07138316B7
:101C10000713831264008A15E819122E071283161F
:101C20000712831264008A1568191A2E8711831609
:101C3000871183128A018D200715831607118312DD
:101C400087148316871064008A15831268182C2E57
:101C5000061383160613831264008A15691A342E3C
:101C6000051283160512831264008A15E81F3C2EA4
:101C7000051483160510831264008A15681E442E0D
:101C800085168316851283128A018D20851483168A
:101C9000851064008A158312681F522E071483165C
:101CA0000710831264008A15E81E5A2E0515831644
:101CB0000511831264008A15E91B622E87108316B2
:101CC0008710831264008A15E91A6A2E0711831699
:101CD000071183128A018D2064008A15691B742EF6
:101CE00085108316851083128A018D208A15542948
:061CF00063008A15782E46
:02400E00D43CA0
:1042E80001001000600000000000A0001000440061
:1042F80002000800C4005000F80014000000440048
:104308000100540000002800020080000300800023
:104318000100C0000000E00000007000000038004C
:0C43280000001C0002000C000300040058
:0643FA00000001000300B9
:00000001FF
